:10F80000000C041E400A040000000000004000003C
:10F810000000000000000000FA70FAE0FB0CFB7929
:10F8200000000140014001400140015409550955C3
:10F83000095509551FFF015401540154015409553C
:10F8400001540154015401541FFF40004000400086
:10F8500040005FFF6E9F00006E9F00026E9F0004DD
:10F860006E9F00066E9F00086E9F000AF878F87879
:10F87000F878FA1DF878F8781A5086011F8B10CEA8
:10F8800001008E0000108EF86CC60CA6A0A7805A4E
:10F8900026F98E0100108EF800C640A6A0A7805A57
:10F8A00026F9CCAA55FD4000B6400081AA2617B61D
:10F8B0004001815526108E012C108EF840C614A6EA
:10F8C000A0A7805A26F99601B720118A10B72013F5
:10F8D000860AB720124FB72021B7202386ECB72025
:10F8E0004C86C0B7204B86F0B7204FB7204386BF69
:10F8F000B72040B72042867FB7204EB7204D86EE16
:10F90000B7204CBDFD808640970DC660B620402BC9
:10F91000FBB620402AFB5A26F34F971043B7280521
:10F92000B728068605B7201286C0B7201086820D3C
:10F930000E2711C60153F728068EFBCD9F1EC60168
:10F94000D7168A01971043B72807BDFC8E1CEF100D
:10F950008E0122BDFD10267E1F894D81DB2611BD43
:10F96000FD1081DC2604C6C0200681DD2602C6DB30
:10F97000BDFD1081DB2611BDFD1081DC260486C093
:10F98000200681DD260286DB9712BDFD1081C02690
:10F990003C96125A26049703202E5A2604970420D8
:10F9A000355A2604970520205A2604970620195A0E
:10F9B0002609910E2705970E7EF92D5A2618847F69
:10F9C0009702961284809700BDFD802009BDFD102E
:10F9D000260481C026F7B6201281052719108E0152
:10F9E00036AE24AC26270F1A10B620128105270444
:10F9F000AD9F011A1CEF0D162F20108E012CAE2486
:10FA0000AC2627161A100D162F0E108E012CAE24C0
:10FA1000AC262704AD9F011E1CEF7EF94FB62011C6
:10FA20002A1585082709AD9F0118B620112A0885D7
:10FA3000102704AD9F011AB62803438501260484CC
:10FA400006271D971185C42706AD9F011C961185B9
:10FA5000322706AD9F011E961185082703BDFC8E37
:10FA6000B6204D2A03BDFCC83B108E0118BDFD0B0E
:10FA7000F6201085072633C1C0262F108E0118BD31
:10FA8000FD0BF62010850726E05D271F12C1C02759
:10FA9000191F984D108E0122BDFD1F26CC108E011E
:10FAA00018BDFD0B108E0122200C39108E0118BDDF
:10FAB000FD0B108E012CF62010850726121F984D85
:10FAC000BDFD1F260A81C026E1AE22AF2420ACAEC8
:10FAD00024AF2281C0269220A2108E011ABDFD0BF8
:10FAE000108E0136BDFD102604B72010398609B7E7
:10FAF0002012108E011ABDFD0B108E0136BDFD10B7
:10FB000026A8C605F72012B7201020CD108E01368A
:10FB1000AE24AF2286C0BDFD1F4F9717BDFD3B1021
:10FB20008E011CBDFD0B8504272C108E0136B628D6
:10FB3000044381C0270881DB260EC6DD2002C6DC17
:10FB400086DBBDFD3B1F984DBDFD3B961185802694
:10FB500009854026B739858027B2108E0136BDFD54
:10FB60004426A986C0BDFD3B0D1726A0AE22AF24BA
:10FB700020A2108E011EBDFD0B86FF97160D0E26CE
:10FB8000399610847F9710860297179E07272B4F70
:10FB900043B728038643BDFCE5DC078EFBB4BDFC00
:10FBA000F4108E011EBDFD0B8502102700914F43FE
:10FBB000B72803398EFBBA9F1E39108E012CBDFD6C
:10FBC0001043B728030D0E26358663202386FF9742
:10FBD0001696108A40971043B7280720578673203F
:10FBE0006DBDFD1026F781C027F743B72803867344
:10FBF000BDFCE5108E011EBDFD0B8520274186430F
:10FC0000BDFCE5108E011EBDFD0B108E012CBDFD4F
:10FC100010263981DB2615BDFD101F894D86C0C118
:10FC2000DC270D86DBC1DD27071F984D81C027B17A
:10FC300043B72803108E011EBDFD0B851027CB1086
:10FC40008E012CBDFD10260481C026F78653BDFC15
:10FC5000E5108E011EBDFD0BDC0B27138EFC6FBD66
:10FC6000FCF4108E011EBDFD0B4F43B728033986EF
:10FC70000197160D0E2614961084BE8A80971043A5
:10FC8000B728070F168640970D8D037EFB72B628A6
:10FC9000020D0E2619438440910D2712970D270F50
:10FCA0000D162B0A0F168620B7204EFC2048390D62
:10FCB0001626FB2007BDFD76D1042307DC098EFC48
:10FCC000B520318601971639FC20480D15270A0A00
:10FCD000154D26015CFD2048398620B7204EB62000
:10FCE000486E9F01209714961084CF9A1497104362
:10FCF000B72807399F2097154F5D26060A152BD97F
:10FD00004353FD204886A0B7204E393510AFA439A3
:10FD1000AE26AC242719A6848D18AF261A0439AE56
:10FD2000221F138D0DAC262706A7C4AF2220ED1C81
:10FD3000FB393001AC282602AEA4398DE2270486B7
:10FD400001971739AE22AC2427E58D0A26EC8D06E3
:10FD500026E8AF2220C68D1026E08D0C26DCA68476
:10FD600081DB27B88DCC20B4ACA42602AE28301F8E
:10FD7000AC2426A820B98615D60F3DCB35D70F3930
:10FD8000C6240D00270158D71296033DDD07D61271
:10FD900096053DDD09D61296063DDD0B0D022604C3
:10FDA00086049702C6604F4CD0022EFB0D00260140
:10FDB0004480022B045FFD204439544E432D3120F2
:10FDC0004B495353206669726D77617265205742C3
:10FDD000364543452C20504130475249203232208D
:10FDE0006465632031393837FFFFFFFFFFFFFFFFF6
:10FDF000FFFFFFFFFFFFFFFFFFFFFFFFFFFFFFFF13
:10FE0000FFFFFFFFFFFFFFFFFFFFFFFFFFFFFFFF02
:10FE1000FFFFFFFFFFFFFFFFFFFFFFFFFFFFFFFFF2
:10FE2000FFFFFFFFFFFFFFFFFFFFFFFFFFFFFFFFE2
:10FE3000FFFFFFFFFFFFFFFFFFFFFFFFFFFFFFFFD2
:10FE4000FFFFFFFFFFFFFFFFFFFFFFFFFFFFFFFFC2
:10FE5000FFFFFFFFFFFFFFFFFFFFFFFFFFFFFFFFB2
:10FE6000FFFFFFFFFFFFFFFFFFFFFFFFFFFFFFFFA2
:10FE7000FFFFFFFFFFFFFFFFFFFFFFFFFFFFFFFF92
:10FE8000FFFFFFFFFFFFFFFFFFFFFFFFFFFFFFFF82
:10FE9000FFFFFFFFFFFFFFFFFFFFFFFFFFFFFFFF72
:10FEA000FFFFFFFFFFFFFFFFFFFFFFFFFFFFFFFF62
:10FEB000FFFFFFFFFFFFFFFFFFFFFFFFFFFFFFFF52
:10FEC000FFFFFFFFFFFFFFFFFFFFFFFFFFFFFFFF42
:10FED000FFFFFFFFFFFFFFFFFFFFFFFFFFFFFFFF32
:10FEE000FFFFFFFFFFFFFFFFFFFFFFFFFFFFFFFF22
:10FEF000FFFFFFFFFFFFFFFFFFFFFFFFFFFFFFFF12
:10FF0000FFFFFFFFFFFFFFFFFFFFFFFFFFFFFFFF01
:10FF1000FFFFFFFFFFFFFFFFFFFFFFFFFFFFFFFFF1
:10FF2000FFFFFFFFFFFFFFFFFFFFFFFFFFFFFFFFE1
:10FF3000FFFFFFFFFFFFFFFFFFFFFFFFFFFFFFFFD1
:10FF4000FFFFFFFFFFFFFFFFFFFFFFFFFFFFFFFFC1
:10FF5000FFFFFFFFFFFFFFFFFFFFFFFFFFFFFFFFB1
:10FF6000FFFFFFFFFFFFFFFFFFFFFFFFFFFFFFFFA1
:10FF7000FFFFFFFFFFFFFFFFFFFFFFFFFFFFFFFF91
:10FF8000FFFFFFFFFFFFFFFFFFFFFFFFFFFFFFFF81
:10FF9000FFFFFFFFFFFFFFFFFFFFFFFFFFFFFFFF71
:10FFA000FFFFFFFFFFFFFFFFFFFFFFFFFFFFFFFF61
:10FFB000FFFFFFFFFFFFFFFFFFFFFFFFFFFFFFFF51
:10FFC000FFFFFFFFFFFFFFFFFFFFFFFFFFFFFFFF41
:10FFD000FFFFFFFFFFFFFFFFFFFFFFFFFFFFFFFF31
:10FFE000FFFFFFFFFFFFFFFFFFFFFFFFFFFFFFFF21
:10FFF000FFFFF854F858F85CF860F864F868F8788F
:0000000000
